:020000040000FA
:02000000812855
:08000800F000030E8301F1007A
:100010000408F2000A08F3000B1919200C194C20EF
:1000200073088A0072088400710E8300F00E700E4F
:1000300009000B11A11A0800A10A2108103A03199E
:1000400037282108033A031D08002208FC39031948
:10005000352809302202031834282208263E84005D
:1000600080308000A20A29282014A2010800F03064
:10007000A6008030A7008030A8008030A900803022
:10008000AA008030AB008030AC008030AD00803002
:10009000AE00A201201408000C118101A101A208E8
:1000A000031D572826308400F03080007228230872
:1000B0001502A300031CA40A24081602A400F730AA
:1000C000A3020030031C0130A402031C7920A40801
:1000D000031D7D202208263E840023088000F03A7C
:1000E000031980031508A3001608A400221EA20A03
:1000F0000800A4010330A3000800A401FD30A30000
:100100000800A001A20183164130810004308C0058
:10011000831260308B0021309000043097008501FD
:10012000860183169B0120308500DF3086000C306D
:100130009900243098008312903098008101A10129
:100140000C110B118B17201CA32820100930A500BF
:10015000263084000C1EAA2800089900840AA50BEA
:04016000AA28A328FE
:02400E00413F30
:02401000FC3F73
:00000001FF
